:103ACF00C2AF53FFBFE4F5F18EF38FF212000AAFCE
:063ADF00F443FF40D2AFEA
:013AE50022BE
:103A9A00C2AF53FFBF75F1A08EF38FF2AF058FF45B
:0B3AAA0012000A43FF40D2AFAFF4222D
:1038AF009062AEEEF0A3EFF0C2AF53FFBF75F180A1
:1038BF0012000A75F1309062AEE0FEA3E0FF8EF3C6
:0E38CF008FF2E4F5F412000A43FF40D2AF225C
:01000A0022D3
:103B5300EEF0A3EFF0E4A3F0A3F022E0FEA3E0FF76
:023B6300C3227B
:1037EA009061FD123B539061FD123B5E906200E0D6
:1037FA009F9061FFE09E501A000000000000000048
:10380A000000906200E004F070DC9061FFE004F0D8
:03381A0080D42235
:10384F009061F9123B539061F9123B5E9061FCE07D
:10385F009F9061FBE09E50177FE87E031237EA903E
:10386F0061FCE004F070DF9061FBE004F080D72290
:10387F009062A6123B539062A6123B5E9062A9E043
:10388F009F9062A8E09E50177F0A7E0012384F90DB
:10389F0062A9E004F070DF9062A8E004F080D72204
:103B6500759850438920438780758BFC758DFCD2F1
:023B75008E229E
:073BCA00C298C299D2AC229F
:083BC2008F993099FDC2992290
:1026E800F090627EE03400F0906274E0FF90626ED9
:1026F800E0FBA3E0FAA3E0F9EF1213C1906275E0E2
:1027080090626EFFE0FBA3E0FAA3E0F92290620971
:10271800E0FEE42401FFEE3440FE22EFF0A3EBF0EC
:10272800A3EAF0A3E9F022906268E0FF90627EE0FD
:10273800FCA3E0AA04F97B00220B906217EBF0A33C
:102748007462F0A37474F0A3E4F0A322FEE42411ED
:10275800FFEE3440FEA3E0FD22900001EF1213D3F8
:10276800906276E09000021213D3906277E09000B6
:10277800031213D3906278E022906209E0FEE42409
:1027880024FFEE3440FE22906209E0FEE42425FF97
:10279800EE3440FE22EFFD7C00E0FEE42DFFEC3E2F
:1027A80022906209E0FEE42428FFEE3440FE2290E5
:1027B8006209E0FEE42429FFEE3440FE22E4F0A39F
:1027C800F0A3F0A3F02225E0249BF582E43461F520
:1027D80083E022E0FF90627CE4F0A3EFF0E0FE22C9
:1027E800906279E07C002400FFEC3E229000030216
:1027F8001394906209E0FEE42404FFEE3440FE22C4
:10280800FFEE3440FE90628622FFEE3440FEA322A3
:10281800E0FDA3E090621CCDF0A3EDF022E0FDA363
:10282800E090621ACDF0A3EDF022FEF0FCA3EFF0E9
:10283800FD22E0F9A3E0FAA3E0906217C922E0FEC6
:10284800E42400FFEE3440FE22E0FFAA04A905902C
:102858006219E4229000010213949000020213947A
:10318F00906209EFF090620BEAF0A3EBF090620A05
:02319F00EDF051
:1031A10064016018E0FF64026012EF6403600DEFD8
:1031B10064046008EF6405600302324A906209E02A
:1031C100FF123A1990620912284690620DE0FD90B3
:1031D100620AE04DFD123B1490620BE0FCA3E04C4F
:1031E100601C1227FAC006C007ECFDD007D00612FA
:1031F10032552405FFEE3440FE90620B802C906224
:10320100B1E004F070069062B0E004F01227FAC059
:1032110006C0079062B0E0A3FDD007D00612325578
:103221002405FFEE3440FE9062B0A3E0FD123B1492
:103231001227157D01123B14122715123A49EF701E
:10324100F790620E7401F08005E490620EF09062D6
:033251000EE0FF8D
:0B32540022123B14906209E0FEE4220D
:103A1900906215EFF01227197D10123B1490621570
:103A2900122718123A49EF70F4906215E0FF7DFFF2
:033A3900023B97B6
:05377D00906209EFF06D
:10378200123B29EF6413701F9062091227187D0201
:10379200123B14906209122718123A49EF70F49002
:1037A200620A7401F08005E490620AF090620AE015
:0137B200FF17
:0137B30022F3
:062C4200906298122723A6
:102C480012137BFFB4FF1890629912270C12285CAC
:102C5800B4FF0C122862B4FF061227F4F46022EFC6
:102C6800701590629912270C12285C700A1228625B
:102C780070051227F4600A90629CE07002A3E0706D
:102C880008E490629EF0022D4090629E7401F090DC
:102C98006298E0FEE4240C12281112270C12137B10
:102CA800122D54240D12281112270C900001122DF8
:102CB80046240E12281112270C900002122D4624C9
:102CC8000F12281112270C1227F4122D542410FF6A
:102CD800EE3440FEC006C00790629CE0A3FDD0071A
:102CE800D006123B14906298E090629C122754120E
:102CF8003B141239369062981227187D04123B143F
:102D0800906298122718123A49EF70F4122D5F64F6
:102D1800156022122D5F6417601B906298E0FF1205
:102D28003BB9EF30E3E6906298E0FF7D08123B97ED
:0D2D3800E490629EF0123AFD90629EE0FF72
:102D450022121394FD123B14906298E0FEE422FDDA
:102D5500123B14906298E0FEE422906298E0FEE453
:0C2D65002403FFEE3440FE123A49EF2236
:103AB500906209EFF01227197D08123B14906209F4
:0A3AC500122718123A49EF70F4229C
:062B080090620912272370
:102B0E0090620F1227C5A3F0A3F0906209E0FE12A7
:102B1E0027CEFCA3E0FD90620DE0FAA3E0FBD39D6F
:102B2E00EA9C4011EE1227CEFDA3E0906213CDF089
:102B3E00A3EDF08008906213EAF0A3EBF090620927
:102B4E00E0FF1235FE906211EEF0A3EFF0122C387A
:102B5E006417600EEF641C6009E4906213F0A3F03A
:102B6E008015906213E0FCA3E0FDC3906212E09D1D
:102B7E00906211E09C40C6122781123A4990620F72
:102B8E00E4F0A3EFF012278F123A49906210122749
:102B9E009D90620F12283290620912285112272737
:102BAE0090621312281890620A12270C122FA79007
:102BBE006213E0FEA3E0FF906210E02FF090620F30
:102BCE00E03EF0122781C006C00790620FE0A3FD21
:102BDE00D007D006123B1412278F90620FA3E0FD90
:102BEE00123B149062091227187D20123B1490623A
:102BFE0009122718123A49EF70F4906209E0FF1299
:102C0E003BB9EF20E411122C3870EF906209E0FF0F
:102C1E00123A19E4FEFF22906209E0FF7D10123B8A
:092C2E0097906213E0FEA3E0FFA1
:0B2C370022906209E0FF123B29EF220F
:06325F0090620912272312
:1032650090620F1227C5D390620EE0940090620D14
:10327500E09400500302331A1227A9123A499062CA
:103285000FE4F0A3EFF01227B7123A49906210123B
:10329500279D90620F122832906209E0FFAA04A9C7
:1032A500057B00C002C001A312283A1227279062AD
:1032B5000D122825D001D0021230A690620DE0FE35
:1032C500A3E0FF906210E02FF090620FE03EF01255
:1032D50027A9C006C00790620FE0A3FDD007D0065E
:1032E500123B141227B790620FA3E0FD123B149016
:1032F50062091227187D40123B14906209122718A3
:10330500123A49EF70F490620DE0FFA3E09062116C
:0D331500CFF0A3EFF0906211E0FEA3E0FF07
:013322002288
:0623A90090628012272360
:1023AF00E490628B1227C6906280E01227CEFEA3C4
:1023BF00E0FF906284E0FCA3E0FDD39FEC9E90626F
:1023CF008B4007EEF0A3EFF08005ECF0A3EDF0905B
:1023DF00628612270C12137B700F12285C700A1280
:1023EF00286270051227F46014906289E07002A3CE
:1023FF00E0600A90628BE07002A3E0700AE49062E2
:10240F008BF0A3F0022523906280E0FEE4240CFF02
:10241F00EE3440FE12137B12253A240D12280812B7
:10242F00270C90000112252C240E12280812270CBD
:10243F0090000212252C240F12280812270C1227A5
:10244F00F412253A2410FFEE3440FEC006C0079068
:10245F006289E0A3FDD007D006122551E090628972
:10246F00122754122551122784123A4990628DE493
:10247F00F0A3EFF0906280122792123A49EFFD7CA1
:10248F000090628E1227A1FE90628D122833906207
:10249F008012285112272790628B12281890628180
:1024AF0012270C122FA790628BE0FEA3E0FF906221
:1024BF008EE02FF090628DE03EF0906280122784C4
:1024CF00C006C00790628DE0A3FDD007D006123B77
:1024DF001490628012279290628DA3E0FD123B143C
:1024EF001239369062801227187D20123B149062A9
:1024FF0080122718123A49EF70F412255820E40F72
:10250F0012255830E3F47D18122545E4FEFF227D95
:0C251F001012254590628BE0FEA3E0FF47
:10252B0022121394FD123B14906280E0FEE422FD14
:10253B00123B14906280E0FEE422906280E0FF1276
:10254B003B97123AFD22123B1490628022906280DC
:07255B00E0FF123BB9EF2283
:06256200906268122723BD
:10256800E490627C1227C6D390626DE0940090627A
:102578006CE0940050030226D79062681227AC12D0
:102588003A4990627EE4F0A3EFF09062681227BAAD
:10259800123A49EFFD7C0090627F1227A190627E7B
:1025A800F0A3EFF0906268122846123A49EF5407F8
:1025B80024FD6053146073240260030226C01227AE
:1025C8002FC0031227417408F0D0031226E0240814
:1025D8001226E812276190627112270BE48FF0121D
:1025E800146E90627112270C12140BFE1227E88FDA
:1025F800F012146E90627A1227DB90627BE024005E
:10260800FFEC3EA302266512272FC0031227417450
:1026180006F0D0031226E024061226E812276112DB
:1026280027DC1227E890627C803312272FC0031220
:1026380027417402F0D0031230A690627FE0240292
:10264800F090627EE03400F09062741227DB9062B2
:10265800751227EBCF24FECF34FF90627CF0A3EFF6
:10266800F012272FC002C00190626912283A12277F
:102678002790627C122825D001D0021230A69062E1
:102688007CE0FEA3E0FF90627FE02FF090627EE0A6
:102698003EF09062681227ACC006C00790627EE0E8
:1026A800A3FDD007D006123B149062681227BA9097
:1026B800627EA3E0FD123B149062681227187D40E9
:1026C800123B14906268122718123A49EF70F4907E
:0726D800627CE0FEA3E0FFBD
:0926DF00221230A690627FE02275
:102E92003D3D3D3D3D3D3D3D3D3D3D3D3D3D3D3D60
:102EA2003D3D3D3D3D3D3D3D3D3D3D3D3D3D3D3D50
:102EB2003D3D3D3D3D3D3D3D3D3D3D3D3D3D0D0AA3
:102EC2000020202020202020573731303041202080
:102ED2004E657420436F6E66696720496E666F7235
:102EE2006D6174696F6E2020202020202020200D2B
:102EF2000A004D4143204144445245535320495016
:102F0200203A20252E3262782E252E3262782E2506
:102F12002E3262782E252E3262782E252E3262785B
:102F22002E252E3262780D0A00252E3362752E254B
:102F32002E3362752E252E3362752E252E33627541
:102F4200005355424E4554204D41534B20203A20C8
:102F520025730D0A00472F572049502041444452FF
:102F6200455353203A2025730D0A004C4F43414CE0
:102F72002049502041444452455353203A2025735E
:102F82000D0A00C0A80102C0A80101FFFFFF000056
:102F920008DC1122330202020202020202020202CF
:052FA200020202020220
:0B3A7D004861AB0000000000000000EA
:10286800906200E025E0FF9061FFE033FE749B2F4B
:10287800F58274613EF58322906200E025E0FF90C6
:1028880061FFE033FE748B2FF58274613EF583227D
:10289800AC02AD03C39DFFEE9CF0A3EFF0A3E0FEF6
:1028A800A3E0FFE422F0A3E4F0747B2FF5827461C7
:1028B8003EF58322F0A3E4F0746B2FF58274613E39
:1028C800F58322FFEE3440FEE0FBA3E0FAA3E0F933
:1028D8008D828C83121394FD123B149061FFE0FCEF
:1028E800A3E0FD227D017BFF7E007F040213552FAC
:1028F800FFE43EFEED34FEFDEC338F0F8E0E8D0DA2
:10290800F50C2225E024B7F582E43461F583E0FE76
:10291800A3E0222FFFE43EFEE434FEFDE433FC2274
:102928007D017BFF7E007F080213557A00AB07E02C
:10293800FEE422E0F510A3E0F51122EFFD7C00EBA8
:10294800FEE42DFBEC3EFA4B228F0F8E0EF50DF5B3
:102958000C22F583E05AFEA3E05FFBAA06E922FEFB
:10296800E42DFFEC3EF0A3EFF022F583E0FCA3E0BA
:10297800C39FEC9E22C2AF7593FE8F828E8322EF97
:10298800F0E4A3F0A3F0FBFA22906209E0FEE4224F
:10299800A3E0FAA3E0FF2225E024C7F582E434612E
:1029A8002225E0249BF582E434612225E0248BF57E
:0529B80082E4346122FD
:103AE600123BD7C2AF123B6575EBFF75ECFF75ED68
:073AF600FF75EEFFD2AF22C5
:101D1D0078317C627A2F79851228EC78357C627A5D
:101D2D002F79891228EC78397C627D017BFF7A2F1F
:101D3D00798D1228F0783D7C627D017BFF7A2F79B9
:101D4D00917E007F0612135578437C627A2F799726
:101D5D00122928784B7C627A2F799F1229287B01D2
:101D6D007A6279391239609062317F0F121F659056
:101D7D0062327F10121F659062337F11121F6D90BA
:101D8D0062347F12121F6D9062357F01121F7590A4
:101D9D0062367F02121F759062377F03121F7D908E
:101DAD0062387F04121F7D123AFD90623D7F091249
:101DBD001F8590623E7F0A121F8590623F7F0B1236
:101DCD001F8D9062407F0C121F8D906241E0FD7F50
:101DDD000D7E00123B14906242E0FD7F0E7E0012DC
:101DED003B149061FC7401F0A37462F0A3744BF08A
:101DFD007B017A627943121FAD121FA37BFF7A2EEE
:101E0D0079C3121A23121FA37F097E00123A49C00B
:101E1D00077F0A7E00123A49C0077F0B7E00123AF7
:101E2D0049C0077F0C7E00123A49C0077F0D7E0026
:101E3D00123A49C0077F0E7E00123A49906211EFA7
:101E4D00F0906210D0E0F090620FD0E0F090620E52
:101E5D00D0E0F090620DD0E0F090620CD0E0F07B1D
:101E6D00FF7A2E79F4121A237B017A627964123982
:101E7D00AC90620C74FFF0A3742FF0A3742BF09050
:101E8D006264E090620FF0906265E0906210F090F5
:101E9D006266E0906211F0906267E0906212F07BF2
:101EAD00017A627953121A1D90620C7401F0A374B9
:101EBD0062F0A37453F07BFF7A2F7943121A237FBC
:101ECD00017E00123A49C0077F027E00123A49C0D6
:101EDD00077F037E00123A49C0077F04121F95D079
:101EED00E0F0906210D0E0F090620FD0E0121F3C55
:101EFD007A2F7957121A237F0F7E00123A49C007A5
:101F0D007F107E00123A49C0077F117E00123A49B8
:101F1D00C0077F12121F95D0E0F0906210D0E0F054
:0F1F2D0090620FD0E0121F3C7A2F796D021A23B9
:101F3C00F090620C74FFF0A3742FF0A3742BF07B61
:101F4C00017A627953121A1D90620C7401F0A37419
:101F5C0062F0A37453F07BFF22E0FD7E00123B1471
:101F6C0022E0FD7E00123B1422E0FD7E00123B14A9
:101F7C0022E0FD7E00123B1422E0FD7E00123B1499
:101F8C0022E0FD7E00123B14227E00123A49906240
:101F9C0012EFF0906211227BFF7A2E7992121A23A3
:011FAC002212
:043BD70075FF402214
:103B770075FE0843FE207F647E0012384F53FEDF38
:013B8700221B
:103B1400A2AFE433FC12297DEDF0E4F593AF04EF9A
:043B240024FF92AF39
:013B2800227A
:0D3A3C00906215E0FEE42420FFEE3440FE11
:103A4900A2AFE433F912297DE0FFE4F593AD01ED6E
:043A590024FF92AF05
:013A5D002246
:093BB900EFFEE42402123A44225A
:0D3B9700EFFEE42402FFEE3440FE023B147A
:0B1FAD009061F9EBF0A3EAF0A3E9F06B
:101FB800E4906201F0A3F0A3F0A3F09061C77480ED
:101FC800F0A3E4F09061B774C0F0A3E4F09061FF6F
:101FD800F0A3F01228E3FEE4241F9061F91228CB45
:101FE800FEE4241E9061FC1228CB25E0FFEC1228A9
:101FF80073E4F0A3F012288DE4F0A3F0C39062011B
:10200800E0648094C050679061F9E0FBA3E0FAA314
:10201800E0F98D828C8312139424FE601D24FE60E7
:102028002624FC602E24F86036240F70411228689C
:1020380074041228AD7403022071122868740812FF
:1020480028AD740702207112286874101228AD7424
:102058000F801612286874201228AD741F800A1287
:10206800286874401228AD743FF0A374FFF0C39041
:102078006203E0648094C050729061FCE0FBA3E0CE
:10208800FAA3E0F9A3E0FEA3E0FFF5828E83121322
:102098009424FE602224FE602B24FC603324F86024
:1020A8003B240F7046EF25E0FFEE12288B740412D4
:1020B80028BC74030220EE12288074081228BC740D
:1020C800070220EE12288074101228BC740F8016A4
:1020D80012288074201228BC741F800A1228807469
:1020E800401228BC743FF0A374FFF01228E325E0E7
:1020F800FFEC122873E0FAA3E0FB906202E02BF0F9
:10210800906201E03AF012288DE0FEA3E0FF9062B1
:1021180004E02FF0906203E03EF0ED4C607B9061AC
:10212800FFA3E025E0FFEC33FE74992FF58274617C
:102138003EF583E0FAA3E0FB74C52FF58274613E97
:102148001229142BFBEE3AFAED25E0FFEC33FE746E
:10215800C72FF58274613EF583EAF0A3EBF074892A
:102168002FF58274613EF583E0FCA3E0FD74B52F82
:10217800F58274613E1229142DFDEE3CFC9062003C
:10218800E025E0FF9061FFE033FE74B72FF582741D
:10219800613EF583ECF0A3EDF0906200E004F0708E
:1021A800069061FFE004F0C3906200E0940890613B
:0B21B800FFE0648094805003021FDBF6
:0121C30022F9
:023B2900AC07E7
:103B2B007BFFECFEE42403123A44EF6B6004AB071B
:023B3B0080F018
:013B3D002265
:0335FE00906215C3
:10360100122987123A3C9062151229332421123A69
:10361100441229436022123A3C906216E4F0A3EF6F
:10362100F0906215E0FEE42421123A44EFFD90622D
:1036310017E0906216122967906216E0FEA3E0FF80
:073641006B7002EE6A70BC21
:01364800225F
:0335AC0090620921
:1035AF001229871229912426123A4490620912296E
:1035BF00332427123A4412294360241229912426D6
:1035CF00123A4490620AE4F0A3EFF01229912427F3
:1035DF00123A44EFFD90620BE090620A1229679055
:0E35EF00620AE0FEA3E0FF6B7002EE6A70B5A8
:0135FD0022AB
:052FA700906215EFF03F
:102FAC00AF01906220EAF0A3EFF090621912299819
:102FBC00906215E0F925E0247BF582E43461122956
:102FCC005A12299F1229142BFFEE3A906222F0A379
:102FDC00EFF090621DE02BFF90621CE03AFEE912CC
:102FEC0029A9122972400302307E906215E0122941
:102FFC00A912291490621E122898FCFDC004C00569
:10300C00C006C0071228A51228F790621E12293B91
:10301C00D007D006D005D00412349290621EE0FE88
:10302C00A3E0FF906221E02FF0906220E03EF0C31D
:10303C0090621DE09FFF90621CE09E90621EF0A3C8
:10304C00EFF0906215E012299FF583E0FFA3E0906A
:10305C006222CFF0A3EFF09062201228A6FCFDC0F4
:10306C0004C005C006C0071228A51228F790621EDE
:10307C0080199062201228A6FCFDC004C005C00671
:10308C00C0071228A51228F790621C12293BD00702
:09309C00D006D005D004123492D4
:0130A5002208
:0E30A600906213EFF0A3EBF0A3EAF0A3E9F0C1
:1030B400A3122998906220EAF0A3EFF09062141210
:1030C4002998906213E0F925E0246BF582E43461D9
:1030D40012295A12290B2BFFEE3A90621EF0A3EF2D
:1030E400F090621BE02BFF90621AE03AFEE912298D
:1030F400B31229725074906213E01229B312291486
:1031040090621C12289812291BC006C0071228A519
:1031140012295190621C12293BD007D00612349216
:1031240090621CE0FEA3E0FF906221E02FF0906229
:1031340020E03EF0C390621BE09FFF90621AE09E85
:1031440090621CF0A3EFF0906213E012290BFF9041
:10315400621EEEF0A3EFF0E412291BC006C00712B2
:1031640028A512295190621C801690621E1228A66E
:1031740012291BC006C0071228A512295190621AF1
:0A31840012293BD007D00612349246
:01318E00221E
:1039600012137B9061B3F09000011213949061B434
:10397000F09000021213949061B5F09000031213BE
:06398000949061B6F022F4
:103936009061B3E0FD7F057E00123B149061B4E018
:10394600FD7F06123B149061B5E0FD7F07123B1424
:0A3956009061B6E0FD7F08023B140B
:103AFD00E4FD7F05FE123B147F06123B147F071277
:073B0D003B147F08023B148A
:1039AC009061B3E01213C19061B4E0900001121366
:1039BC00D39061B5E09000021213D39061B6E09001
:0539CC0000030213D30B
:103492008F0B8E0A8D098C08A2AFE433F514859345
:1034A20015781012149EA907AF0FAE0EAD0DAC0C1D
:1034B200781012149EAB07C2AFE5111511AE107051
:1034C2000215104E6022899378081214E18F828EC1
:1034D20083E0751200F5138B93AA13780C1214E192
:1034E2008F828E83EAF080D1E51424FF92AF851596
:0234F200932223
:1029BD000D0A414343455320492F4F2050726F64F8
:1029CD00756374732C20496E632E0D0A4D6F64650B
:1029DD006C204554482D44494F2D3438204669729A
:1029ED006D77617265205265766973696F6E20250A
:1029FD00782E2578206275696C643A257320402005
:102A0D002573200D0A0030382F32372F3138003022
:102A1D00383A34373A3234004D4143204144445220
:102A2D0045535320495020202020203A20252E3276
:102A3D0062782E252E3262782E252E3262782E2542
:102A4D002E3262782E252E3262782E252E32627825
:102A5D000D0A00252E3362752E252E3362752E2517
:102A6D002E3362752E252E33627520005355424E3E
:102A7D004554204D41534B20202020202020203A2A
:102A8D002025730D0A0047617465776179204950DF
:102A9D002041444452455353203A2025730D0A00DA
:102AAD00495020414444524553532020202020209A
:102ABD002020203A2025730D0A004F505431203D1F
:102ACD002025632020202020004F505432203D200F
:102ADD0025630D0A0049502041444452455353206B
:102AED00202020203A2025730D0A00080201010143
:0B2AFD000101010802010101010101BB
:053A88004200000000F7
:0B3BA4007D017BFF7E007F08021355AF
:033BDB00C2B7224C
:033BDE00D2B72239
:10163C0078E97C617A2A79F8123BA478F17C617A9A
:10164C002B7900123BA4E4902105F0902104F012B8
:10165C003AE69061FC7401F0A37461F0A374F1F0AC
:10166C007B017A6179E9121FAD75FF28E4F59DF5D0
:10167C009E759203758E02759C3F1234F490620C29
:10168C007401F0A37422F0A374FFF0A3742AF0A3E6
:10169C007413F0A374FFF0A3742AF0A3741CF07BF2
:1016AC00FF7A2979BD121A237F097E00123A49C0AC
:1016BC00077F0A7E00123A49C0077F0B7E00123A60
:1016CC0049C0077F0C7E00123A49C0077F0D7E008F
:1016DC00123A49C0077F0E7E00123A49906211EF10
:1016EC00F0906210D0E0F090620FD0E0F090620EBB
:1016FC00D0E0F090620DD0E0F090620CD0E0F07B86
:10170C00FF7A2A7925121A237F057E00123A49C0E6
:10171C00077F067E00123A49C0077F077E00123A07
:10172C0049C0077F08121971D0E0F0906210D0E028
:10173C00F090620FD0E01218FB7A2A7979121A23F2
:10174C007F017E00123A49C0077F027E00123A499F
:10175C00C0077F037E00123A49C0077F041219713B
:10176C00D0E0F0906210D0E0F090620FD0E0121850
:10177C00FB7A2A7993121A237F0F7E00123A49C002
:10178C0007121990C007121998C007121961D0E0FE
:10179C00F0906210D0E0F090620FD0E01219247A31
:1017AC002A79AD121A232089047F0180027F0090D0
:1017BC0061D7EFF07A2A79C71219A0208B047F0128
:1017CC0080027F009061D7EFF07A2A79D61219A0A7
:1017DC009001027401F07A007B027DE17CCAE4FF87
:1017EC00120D697F0112194D7F021208007F03123E
:1017FC00194D7F041219AC7F051219AC7F06120823
:10180C0000123709902103E0602A14F07F017E005A
:10181C0012384F902103E0701B7B017A4179321210
:10182C0036CC7B017A41793612368F7B017A41793D
:10183C003A1237B4308B33902105E0702D123649B3
:10184C0012197FC007121990C007121998C00712FD
:10185C001961D0E0F0906210D0E0F090620FD0E00F
:10186C001219247A2A79E2121A23208B05E490218A
:10187C0005F030896C902104E0706612390A121957
:10188C007FC0077F107E00123A49C0077F117E008F
:10189C00123A49C0077F127E00123A49906212EF49
:1018AC00F0906211D0E0F0906210D0E0F090620FF6
:1018BC00D0E0F090620C74FFF0A3742AF0A3746073
:1018CC00F07B017A6179D8121A1D90620C7401F0C8
:1018DC00A37461F0A374D8F07BFF7A2A79E2121A10
:0F18EC00233089030217E2E4902104F00217E28F
:1018FB00F090620C74FFF0A3742AF0A37460F07B79
:10190B00017A6179D8121A1D90620C7401F0A374DC
:10191B0061F0A374D8F07BFF22F090620C74FFF09F
:10192B00A3742AF0A37460F07B017A6179D8121A40
:10193B001D90620C7401F0A37461F0A374D8F07B5A
:10194B00FF227A017B037DE07CCA1208007A017BBF
:10195B00037DE07CCA227F127E00123A499062120C
:10196B00EFF0906211227E00123A49906212EFF072
:10197B00906211227B017A4179321236CC7F0F7E35
:10198B0000123A49227F107E00123A49227F117EC3
:10199B0000123A49227BFF243090620CF0121A237A
:0D19AB00221208007A017B037DE07CCA2235
:10370900900000E07002A3E0601A90000074FFF5D9
:10371900F01213F5FEC3E5F09440EE6480948050F6
:103729001A023BDB900102E06011900000E4F0A373
:0B3739007480F0123BDEE4900102F00F
:013744002262
:03002300023BD1CC
:063BD100309802C2983298
:10355200906207E0FBA3E0FAA3E0F9229001027473
:1035620001F09041267482F0A3F0A3F0A3F0E4A34B
:10357200F022EBF0A3EAF0A3E9F012137BFD227430
:10358200C0F074A8A3F0A37401F022904145F07B2F
:10359200017A41792622900003121394FD229000B1
:0A35A200010213949000020213943A
:0B374500906207EBF0A3EAF0A3E9F0AC
:10375000E4A3F090620AE0FD2409FFE433FE9062E6
:10376000071235558D82758300121394FD123B1498
:0C37700090620AE004F0E0C3940640D729
:01377C00222A
:1037B4009062071235747F017E00123B1412355259
:1037C4001235A0FD7F027E00123B141235521235D1
:1037D400A6FD7F037E00123B141235521235987FEA
:0637E400047E00023B140C
:10368F009062071235747F057E00123B149062071B
:10369F001235551235A07F061236C2123555123526
:1036AF00A67F071236C21235551235987F087E0055
:0D36BF00023B14FD7E00123B1490620722B6
:1036CC009062071235747F0F7E00123B14906207D4
:1036DC001235551235A07F101236FF1235551235A2
:1036EC00A67F111236FF1235551235987F127E00C7
:0D36FC00023B14FD7E00123B149062072279
:10390A0012355EA3F0904132123581A374AEF0A352
:10391A0074FF12356BA3123581745E123586E41278
:0C392A00358D123A5E9021047401F022E9
:1036490012355EA3F0A3F0A37408F0A374DCF0A311
:103659007411F0A37499F0A37477F0A3740AF0A31A
:103669007401F0A3F0A374FBF0A374FF12356BA3EC
:10367900740AF0A3740112356B12358D123A5E90FB
:0636890021057401F0228E
:1034F400123591123BAF904126E0FFB48203308B2A
:1035040005123649802430890512390A801C9041FD
:103514002AE0B40106A3E06422600F90412A7401FA
:10352400F0A37422123590123A5E7B017A4179320B
:103534001236CC7B017A41793A1237B47B017A4155
:0E354400793612368F7B017A41792C02374599
:103B3E00AE028EFB8FFAE4FBFDFC22EBF0A3EAF063
:053B4E00A3E9F0E422F0
:1038DD00E490620AF0A2AF33F0C2AF53FFBF8FF195
:1038ED00AE04AF058EF38FF2AF038FF41207FD43D5
:0C38FD00FF4090620AE024FF92AFAFF49D
:01390900229B
:103A5E00906207123B49FBFDFC7FD01238DD90626D
:0F3A6E0007A3E0FAA3E0FF123B3E7FD10238DD51
:0A3BAF00AF01123B3E7FD20238DD69
:1039D100AC02AD018CFB8DFA9062A4E0FCA3E0295E
:1039E100F9EA3CAD01F5FD8DFCAD07AC06E4FB7FCA
:0439F100A10238DD1A
:0934240090628FEEF0A3EFF0A31B
:10342D00123B49906296F0A3F0906294E0FEA3E007
:10343D00FFA3E0FCA3E0FDC39FEE6480F8EC648085
:10344D00985041906290E02DFF90628FE03CCF2428
:10345D00FFCF34FF8F82F583740193FF906291E06B
:10346D00FBA3E0FAA3E0F9906296A3E0F5828C83CA
:10347D00EF1213D3906297E004F070AD906296E076
:04348D0004F080A522
:013491002218
:10700000C2AF75FF407F717E001271D17F617E003B
:107010001271D1E4900000F0A3F0FFFE1271B77F6F
:10702000007E681271B753FFBF75F18012000A75B8
:10703000F130900000E0FEA3E0FF8EF38FF2E4F564
:10704000F412000A43FF401271AF53FFBF75F1A065
:10705000900000E0FEA3E0FF8EF38FF2E42FF582B4
:1070600074803EF583E0F5F412000A43FF4090007F
:1070700001E004F07006900000E004F0D3900001FD
:10708000E09400900000E0946840097F317E001297
:1070900071D1800C900000E05403FEA3E04E70AA72
:1070A000A2A2B392A2A2A3B392A3C3900000E094C1
:1070B0006850030270267F427E001271D1E4900076
:1070C00000F0A3F01271AFC20020003853FFBFE4FC
:1070D000F5F1900000E0FEA3E0FF8EF38FF21200C6
:1070E0000AAFF443FF40900000E0FCA3E0FDE42D74
:1070F000F58274803CF583E06F6009D2007F437EA7
:10710000001271D1900001E004F07006900000E0E0
:1071100004F0D3900001E09400900000E0946840F7
:10712000097F327E001271D1800C900000E0540380
:10713000FEA3E04E7093C200A2A2B392A2A2A4B397
:1071400092A4C3900000E0946850030270C4C2A2ED
:10715000D2A3D2A47F7A7E001271D1020000AD07C3
:10716000EDC4540FFFC3940A400BEF75F00A84E599
:10717000F02441800CEDC4540F75F00A84E5F0242E
:1071800030FFE433FE1271D1ED540FFFC3940A4077
:107190000BEF75F00A84E5F02441800BED540F7578
:1071A000F00A84E5F02430FFE433FE1271D122901E
:1071B0000000E0FEA3E0FFAB07AA06EAFF12715E43
:1071C000AF0312715E7F0D7E001271D17F0A0271D2
:0971D000D18F993099FDC299227A
:102D71000D0A4143434553204554482D44494F2DA5
:102D810034382055706C6F616420506F7274204329
:102D91006F6E6E65637465640D0A0055706C6F61CA
:102DA1006420446174616772616D3A2025730D0A74
:102DB100005374617475733D382C206C696E656CB9
:102DC100656E6774683D25303262782066756C6C7B
:102DD100646174616772616D3D2530326278206390
:102DE1006F6D706172653D25303262780053746198
:102DF1007475733D31302C206C696E656373756D2C
:102E01003D2530326278206373756D5F63616C6359
:102E11003D25303262782C2073756D3D253032624C
:102E210078200D0A006C61756E6368696E672066B3
:102E31006C61736820636F7079206F706572617463
:102E4100696F6E2066726F6D20253034780D0A002F
:102E51000D0A666C61736820636F70792072657406
:102E610075726E65643F213F21213F20756E657843
:102E71007065637465642073686F756C6420686144
:102E8100766520637261736865642E2E2E2E0D0A9D
:012E91000040
:0C3A8D00414146004141470041414800D2
:1021C4002406F582E43EF583E0FD7F007E80123B29
:1021D400889061FCE0FEA3E02407F582E43EF583E9
:1021E400E0FD7F017E80123B889061FCE0FEA3E06D
:1021F4002408F582E43EF583E0FD7F027E80123BF5
:10220400889061FCE0FEA3E02409F582E43EF583B6
:10221400E0FD7F037E80123B889061FCE0FEA3E03A
:10222400240AF582E43EF583E0FD7F047E80123BC0
:10223400889061FCE0FEA3E0240BF582E43EF58384
:10224400E0FD7F057E80123B88906202E0FBA3E004
:10225400FAA3E0F974051213C1906202E0FBA3E053
:10226400FAA3E02274049000051213D39061F9E0FC
:102274009061FCFFE0FCA3E090620DAA04F97B01ED
:10228400E4F0A322F9900005121394904132F090E7
:102294000006121394904133F090000712139490A7
:1022A4004134F09000080213949001027401F0226A
:1022B4009061F9E09061FCFFE0FCA3E0AA04F97BE3
:1022C40001A3E0FDA3E090620DCDF0A3EDF022FAAE
:1022D400A90790620C7401F0A3EAF0A3E9F022F9D3
:1022E400906200E0FEA3E0FF22F9E43AFA0D023A1C
:1022F40009904150E0906200FFE0FCA3E0FDC39F21
:10230400EC2212137BFFFD3395E0FC906166E02D17
:10231400F0906165E03CF022F9900005021394EE20
:10232400F0A3EFF0D39400EE940022E0FFA3E0FAD0
:10233400A3E0FB90620D7420F07D0122E02430F0D4
:10234400906165E03400F022EFF0A3ECF0A3EDF02F
:10235400A3EAF0A3EBF0F922F99000010214B1F022
:10236400900006021394F09000070213942DFD9040
:1023740061FCE03400FAA9057B0122F09000090217
:102384001394F090000A021394F912137BFFC364B0
:102394008094C122F582E43EF58322E0FF9061FC43
:0523A400E0FCA3E022B3
:043B88008F828E8317
:0A3B8C00AF05759301EFF0E4F59327
:013B9600220C
:1039F500FDE43EFCE92DF9EA3CFAE42FFFEE3480C4
:043A0500FEAD07FC0F
:043A09008D828C839B
:0C3A0D00759301E0FFE4F593EF0213C194
:030800009061F90B
:1008030012234C9062021222D99061F9E0FF123B4D
:1008130029EF7003020D0624ED7003020D1724F770
:100823007003020CFE24056003020D1F9061F9E0C2
:08083300FF123BB9EF30E05762
:10083B00E4906205F0906205E0FFC39407503E9090
:10084B0061F9E0FEEF6E602D906205E0FF123B292F
:10085B00BF1722E49061FEF0A3F0906205E0FF90D9
:10086B0061FCE0FCA3E0AA04F97B01E490620DF0CB
:10087B00A3F0122B08906205E004F080B89061F9A8
:07088B00E0FF7D01123B9725
:100892009061F9E0FF1235AC9061FE122323500300
:1008A200020D1F9061F9E09061FC1222BB12325FCF
:1008B2009061FEEEF0A3EFF012225D12235C12159E
:1008C200250B05436847570AAB4368494F0ADE4385
:1008D2006849500C0843684D430B7743684E500BF0
:1008E2007743684E570B3E4368534D092744494F9F
:1008F200210A4E524144490CDE525044490C5B528B
:100902005374610CBE554461740CC25546696E093C
:10091200405741444F09605750444F096057525065
:100922004400000CDE1222AD12224DF99000011299
:1009320015015F4572729000057432020AD61222C6
:10094200AD9061FCE0FEA3E01221C4F99000011217
:100952001501575F4F4B9000057406020AD612220A
:08096200ADE4906200F0A3F087
:10096A001222E4240CFDE43EFC9061FCE0FAA3E0D0
:10097A00FB2DF582EA3CF583E0F9906205F0EF245D
:10098A0006FFE43EFEEB2FF582EA3EF583E0906235
:10099A0006F0FEE95E906205F0EEF4A3F012225D25
:1009AA001222E3240C1239F512225D1222E3240CDE
:1009BA00122398121394FD906206E05DFD90620581
:1009CA00E04DFDF0E42FFFEE3480FE123B88122248
:0909DA005D1222E324061239F536
:1009E300906201E004F07006906200E004F0C390AE
:1009F3006201E09406906200E09400500302096AE9
:100A030012225D12235C7B4F7A4479507857C312CC
:100A1300148D9062027016122250F9900001121583
:100A230001575F4F4B9000057406020AD6122260ED
:100A3300F9741112225AF9900001121501525F4FF5
:100A43004B740C12226A7412020CFA1222AD122297
:100A53005DF9740B12225AF9900001121501525FCD
:100A63004F4B90000574061213D3E92406F9E43AB8
:100A7300FA7D007C80123A0912225D24071222EDCE
:100A830012225D24081222ED12225D24091222EDA6
:100A930012225D240A1222ED12225D240B1222ED92
:100AA300122270740C020CFA1222ADC2B69061FCD1
:100AB300E0FEA3E0FF240D122398E0543FF5B0EFCE
:100AC3001221C4F9900001121501575F4F4B90009A
:100AD30005740612226D7406020CFA1222AD12225C
:100AE3005D122288904135F0122258F990000112CC
:100AF3001501575F4F4B122268120D20120D4B0246
:100B03000C051222AD12225D12231C90413A1223CE
:100B13006390413B12236A90413C1222A690413DCF
:100B2300F0122258F9900001121501575F4F4B1232
:100B33002268120D20120D55020C051222AD12224D
:100B43005D12231C90413612236390413712236AAE
:100B53009041381222A6904139F0122258F99000A0
:100B630001121501575F4F4B122268120D2F120D00
:100B73005F020C521222AD12225D1222889041357F
:100B830012237F904136122386904137F090000B59
:100B9300121394904138F090000C12139490413941
:100BA300F090000D12139490413AF090000E12133E
:100BB3009490413BF090000F12139490413CF090BD
:100BC300001012139490413DF0122258F990000145
:100BD300121501575F4F4B122268120D2F12225D1F
:100BE30012235C7B577A4E79687843C312148D7055
:100BF3000B120D4B120D5F120D55800690210374DD
:100C030064F0020C521222AD12225D12231C904199
:100C13002C12236390412D12236A90412E1222A697
:100C230090412F12237F904130122386904131F05F
:100C3300122258F9900001121501575F4F4B1222EF
:100C4300687406120D3E7B017A41792C1237457B7D
:100C5300017A417926023A5E1222AD12225DF974BD
:100C63002412225AF9900001121501525F4F4BE4EE
:100C7300906200F0A3F01222E47B012426F9744170
:100C83003EFA12137BFD12225D2405F9E43AFAE9D8
:100C93002FF9EA3EFAED1213C1906201E004F070FD
:100CA30006906200E004F0906200E07004A3E06448
:100CB3002070C31222707425020CFA1222AD221284
:100CC30022AD12224DF9900001121501575F4F4BCF
:100CD300900005E412226D7406801C1222AD1222CC
:100CE3005DF9740412225AF99000011215015F454F
:100CF30072721222707405120D3E229061F9E0FFA8
:100D0300023AB59061F9E0FF123A199061F91223A2
:0C0D13002F02318F9061F9E0FF12377D54
:100D1F00227406F0122B089061FEEEF0A3EFF02282
:100D2F007406F0122B089061FEEEF0A3EFF022F0A4
:100D3F00122B089061FEEEF0A3EFF0227B017A41B7
:100D4F0079321236CC227B017A41793A1237B422AA
:0A0D5F007B017A41793612368F22AB
:1033AF00E490620CF0A3EB1222DB12230612398693
:1033BF00501990620D12226012238D5005EF24D008
:1033CF00800512137B24C990620CF090620EE47595
:1033DF00F0011213F590620D122260F9122306907C
:1033EF00620CE0FEC454F0F0123986501C90620D4E
:1033FF0012226012238D5005EF24D0800512137B0B
:10340F0024C9FF90620CE02FF090620CE0FF9061F6
:04341F0069E02FF041
:013423002286
:10381D00906209EB1222DB9062091222602402F9F8
:10382D00E43AFA1233AF7E00C006C0079062091267
:10383D002260F91233AFEFFCD0E02400FFD0E03C62
:02384D00FE2259
:030D69009061F99D
:100D6C0012234C9062021222D9A31222D9E4A3F0CE
:100D7C009061F9E0FF123B29EF700302123424ED6D
:100D8C00700302124524F7700302120E240560034F
:100D9C0002124D9061F9E0FF123BB9EF30E0189070
:100DAC0061F9E0FF7D01123B97E4904146F07BFF37
:100DBC007A2D7971121A2312124E12232850030223
:100DCC000E60904146E070299061F912239F906269
:100DDC000D12227F0412125F9061FCE0FEA3E0F57D
:100DEC00828E83E0904147F09041467401F0020EF0
:100DFC0060904147E0FFD39061FFE09F9061FEE07F
:100E0C0094009061F9E0FF904146E0FD9061FDE0B7
:100E1C0050101223719061FEE0FDA3E090620DCDA5
:100E2C00800C122371904147E0FD90620DE4F0A319
:100E3C00ED12125F9061FEA3E0FF904146E02FF0AF
:100E4C00A3E0C39FF0700D904146E0906208F0E47F
:100E5C00904146F0906208E0700302120890620222
:100E6C0012226012235C1215250F06554461741171
:100E7C005F5546696E0E8B55706C6400001208123B
:100E8C0022ADE4904147F0A3F0A3F0906169F0909B
:100E9C006165F0A3F090414EF0A3F0906163F0A374
:100EAC00F090414CF0A3F074FF90414AF0A3F09005
:100EBC0041487401F0A3122363FE12231D7C00240D
:100ECC0000FFEC3E90414EF0A3EF1222A6FE12233F
:100EDC006B2400FFEC3E4F60069041497420F0906B
:100EEC006202122260F9122387FE1223807C0024F6
:100EFC0000FFEC3E9061670212041222AD90414853
:100F0C00E064016003021208A3E0FF6401600302C5
:100F1C00115790620512226012231C643A6008EF8C
:100F2C004402904149F022906166E0243A12234336
:100F3C0090000C12143664307004E5F064306008D4
:100F4C00904149E04404F022906166122340A312C0
:100F5C0023409062051222602406F9E43AFA123317
:100F6C00AF904150EFF09062051222602408F9E432
:100F7C003AFA12381D906161EEF0A3EFF0904150F7
:100F8C00E0F92FFFE43ECF24FFCF34FFFEC39041A6
:100F9C004DE09F90414CE09E5005EEF0A3EFF09099
:100FAC00414AE0FEA3E09061611222FC9E50089041
:100FBC00414AECF0A3EDF0906208E0FD24F0FBE474
:100FCC0034FFFAE975F002A46B7003E5F06A603C3B
:100FDC00904149E04408F09061FCE0FEA3E0FF2D55
:100FEC00122398E4F0EF2405FFE43E1222D31212F0
:100FFC00797A2D79B2904150E025E090620CF09016
:10100C006208E090620DF024F00210C7E4906200D8
:10101C00F0A3F01222F59400503E9062051222606B
:10102C00240EF9E43AFAED25E0FFEC33FEE92FF952
:10103C00EA3EFA1233AF906200E0FCA3E02451F5D3
:10104C008274613CF583EFF0906201E004F070C3B0
:10105C00906200E004F080BB906205122260240EC6
:10106C00F9E43AFA904150E075F002A429F9EA3516
:10107C00F0FA1233AF90616AEFF0906169E0604072
:10108C00904149E04410F090620812239FFD2FF527
:10109C0082E43CF583E4F0ED2405FFE43C1222D31A
:1010AC001212797A2D79EE90616AE0FF90620CF061
:1010BC00906169E0FE90620DF0EF2EA3F0021A230E
:1010CC00906164E004F07006906163E004F090417C
:1010DC004EE0FEA3E0FF906163E0B5062AA3E0B505
:1010EC000725904149E054FEF0906165E0FEA3E0D5
:1010FC00FF906168E02FFF906167E03E4F600890C1
:10110C004149E04440F022E4906200F0A3F0122246
:10111C00F59400400302120874512DF58274613C61
:10112C00F583E0FF906162E02DFD906161E03CFC95
:10113C00E42DF58274803CF583EFF0906201E004BD
:10114C00F070CB906200E004F080C3904149E04421
:10115C0080F0221222ADE4904148F0A3E0906202AC
:10116C00704B122260F974041213C19062021222A5
:10117C0060F9900001121501575F4F4B9061F9E037
:10118C009061FC122277740512126CC2AF7BFF7A4D
:10119C002E792690620C7470F0A3E4F0121A2312CC
:1011AC0070007BFF7A2E7951121A23803412226040
:1011BC00F974051213C1906202122260F9900001B9
:1011CC001215015F457272904149E09000051213AF
:1011DC00D39061F9E0FF9061FC1222787406121230
:1011EC006CE4904146F012124E122328400E12224B
:1011FC00B412325F9061FEEEF0A3EFF0E49062085F
:10120C00F0229061F9E0FF1235AC9061FE122323BD
:10121C00400E1222B412325F9061FEEEF0A3EFF09A
:10122C009061F9E0FF023AB59061F9E0FF123A19CA
:10123C009061F912232F02318F9061F9E0FF123780
:01124C007D24
:10124D00229061F9E0FF1235AC9061FEEEF0A3EF54
:10125D00F022F012325F9061FEEEF0A3EFF022F07B
:10126D00122B089061FEEEF0A3EFF0227BFF7A2D9A
:08127D00799C121A237BFF2269
:03000000023323A5
:0C332300787FE4F6D8FD75812102336A42
:10128500E709F608DFFA8046E709F208DFFA803E4B
:1012950088828C83E709F0A3DFFA8032E309F60838
:1012A500DFFA8078E309F208DFFA807088828C83A0
:1012B500E309F0A3DFFA806489828A83E0A3F60854
:1012C500DFFA805889828A83E0A3F208DFFA804C2E
:1012D50080D280FA80C680D4806980F28033801005
:1012E50080A680EA809A80A880DA80E280CA80336E
:1012F50089828A83ECFAE493A3C8C582C8CCC583E6
:10130500CCF0A3C8C582C8CCC583CCDFE9DEE780B5
:101315000D89828A83E493A3F608DFF9ECFAA9F034
:10132500EDFB2289828A83ECFAE0A3C8C582C8CC8A
:10133500C583CCF0A3C8C582C8CCC583CCDFEADEA3
:10134500E880DB89828A83E493A3F208DFF980CC05
:1013550088F0EF60010E4E60C388F0ED2402B404FE
:101365000050B9F582EB2402B4040050AF232345A5
:0613750082239012D573E3
:10137B00BB010689828A83E0225002E722BBFE0270
:09138B00E32289828A83E49322A3
:10139400BB010CE58229F582E5833AF583E022500E
:1013A40006E92582F8E622BBFE06E92582F8E22258
:0D13B400E58229F582E5833AF583E4932272
:1013C100BB010689828A83F0225002F722BBFE010B
:0213D100F32205
:1013D300F8BB010DE58229F582E5833AF583E8F050
:1013E300225006E92582C8F622BBFE05E92582C8FC
:0213F300F222E4
:1013F500C5F0F8A3E028F0C5F0F8E5821582700283
:061405001583E038F0221F
:10140B00BB010A89828A83E0F5F0A3E022500687AC
:10141B00F009E71922BBFE07E3F5F009E31922896E
:0B142B00828A83E493F5F074019322A1
:10143600BB0110E58229F582E5833AF583E0F5F0F4
:10144600A3E0225009E92582F886F008E622BBFED1
:101456000AE92582F8E2F5F008E222E5832AF58317
:08146600E993F5F0A3E99322DC
:10146E00BB010A89828A83F0E5F0A3F0225006F7C9
:0F147E0009A7F01922BBFE06F3E5F009F31922C6
:10148D00EB9FF5F0EA9E42F0E99D42F0E89C45F0B5
:01149D00222C
:10149E00E8600FECC313FCED13FDEE13FEEF13FF2C
:0314AE00D8F12250
:1014B100BB010DE58229F582E5833AF58302156BBF
:1014C1005007E92582F802155FBBFE07E92582F87E
:1014D100021577E58229F582E5833AF583021583C2
:1014E1007401FF3395E0FEFDFC080808E6CF2FF6F6
:1014F10018E6CE3EF618E6CD3DF618E6CC3CF622CF
:10150100BB010DE58229F582E5833AF5830215AC2D
:101511005007E92582F8021593BBFE07E92582F8F9
:041521000215DD22B0
:10152500D083D082E4937012740193700DA3A393BA
:10153500F8740193F5828883E4737402936C7012D6
:101545007403936D700C7404936E70067405936F39
:0A15550060DDA3A3A3A3A3A380CA33
:1019B800E508240CF582E43462F583E005082290FA
:1019C800620930070390620CE475F0011215F60203
:1019D800137B2000E97F2ED2008018EF540F24904B
:1019E800D43440D4FF30040BEF24BFB41A005003A2
:1019F8002461FFE50960021509050CE50C70020574
:101A08000B30070E906209E475F0011215F6EF022B
:101A180013C1023BC27403D2078003E4C207F5086E
:101A280090620912160DE4F509F50BF50CE509604D
:101A3800077F201219FB80F5750AFFC201C200C298
:101A480002C203C205C206C2081219C7FF700D30D0
:101A580007057F00121A0CAF0CAE0B22B4255FC22B
:101A6800D5C2041219C7FF24D0B40A00501A75F061
:101A78000A780930D50508B6FF0106C6A426F6205F
:101A8800D5047002D20380D924CFB41A00EF5004D1
:101A9800C2E5D204021C0DD20180C6D20080C0D299
:101AA8000280BCD2D580BAD20580B47F201219FB3F
:101AB8002002077401B5090040F11219B8FF121984
:101AC800FB021A35D208D20680951219B8FB1219F2
:101AD800B8FA1219B8F94A4B700679DE7A1C7BFFFE
:101AE80020022EE509602A7E008E8275830012137B
:101AF8009460060EEE650A70F0C2D5EBC0E0EAC04D
:101B0800E0E9C0E0EE121C54D0E0F9D0E0FAD0E0F1
:101B1800FB12137BFF60AAEBC0E0EAC0E0E9C0E07B
:101B28001219FBD0E02401F9D0E03400FAD0E0FB30
:101B3800E50A0460DCD50AD980877BFF7A1C7950D6
:101B4800D202809C791080027908C206C2088008F7
:101B5800D2D5790A8004790AC2D5E50A047002F55B
:101B68000AE4FAFDFEFF1219B8FC7B0820011312E3
:101B780019B8FD7B1030000A1219B8FE1219B8FF07
:101B88007B20EC3382D592D55013C3E43000069FF6
:101B9800FFE49EFEE42001039DFDE49CFCE4CBF8F9
:101BA800C201EC700CCFCECDCCE824F8F870F380ED
:101BB80017C3EF33FFEE33FEED33FDEC33FCEB33AD
:101BC800FB994002FB0FD8E9EB300105F8D0E0C4DF
:101BD80048B201C0E00AEC4D4E4F78207B0070C23D
:101BE800EAB50A0040BCC0E0121C56D0F0D0E02094
:101BF8000104C4C0E0C4B201C0F01219E4D0F0D5A9
:101C0800F0EB021A351216161AD2531B4C581AA3A7
:101C18004C1A9F421B504F1B58441B58491AB84333
:081C28001B5E551B42461B42E6
:101C3000451B42471CFE501AA72D1AAB2E1ACE2B5D
:101C40001AAF231ACC201CE72A1A674800001AC6CC
:101C50003F3F3F00790AA2D5200314300509B9108F
:101C6000020404B9080104A2D52006025001042090
:101C700002689202B509005034C0E07F2030031999
:101C80007F30A20272067205500F121CADC202C252
:101C900006C205C2087F30800F300503E9C0E0129C
:101CA00019FB300503D0E0F9D0E0B509CC300517B9
:101CB0007F30B9100C1219FB7F583004077F7880F1
:101CC00003B908031219FB3002057F2D0219FB7FAF
:101CD000202008F87F2B2006F322920280CF286E66
:101CE000756C6C2900D2011219B83001F8C2017864
:101CF0000930D50108F6021A672D504349581219C8
:101D0000B82403B405004001E4901CF9931219ECC7
:0D1D1000743A1219ECD203750904021B4C41
:10398600EFC394414005EF94474016EFC39461405E
:1039960005EF9467400BEFC394304008EF943A501C
:0639A60003D38001C322DF
:10332F0002163CE493A3F8E493A34003F68001F262
:10333F0008DFF48029E493A3F85407240CC8C3339F
:10334F00C4540F4420C8834004F456800146F6DF6E
:10335F00E4800B0102040810204080903A7DE47E47
:10336F00019360BCA3FF543F30E509541FFEE49363
:10337F00A360010ECF54C025E060A840B8E493A32A
:10338F00FAE493A3F8E493A3C8C582C8CAC583CA55
:10339F00F0A3C8C582C8CAC583CADFE9DEE780BE0D
:013A9900002C
:0C155F00E6FC08E6FD08E6FE08E6FF22B8
:0C156B00E0FCA3E0FDA3E0FEA3E0FF22F3
:0C157700E2FC08E2FD08E2FE08E2FF22B0
:10158300E493FC740193FD740293FE740393FF22AE
:10159300D083D082E493F608740193F6087402931F
:0915A300F608740393F674047356
:1015AC00A8828583F0D083D0821215C31215C31282
:1015BC0015C31215C3E473E493A3C583C5F0C583A7
:1015CC00C8C582C8F0A3C583C5F0C583C8C582C889
:0115DC0022EC
:1015DD00D083D082E493F208740193F208740293DD
:0915ED00F208740393F274047314
:1015F600F8E0FBA3A3E0F925F0F0E582158270027E
:071606001583E0FA38F02221
:09160D00EBF0A3EAF0A3E9F022DE
:10161600D083D082F8E4937012740193700DA3A363
:1016260093F8740193F5828883E473740293686077
:06163600EFA3A3A380DF77
:00000001FF
